:020000040000FA
:02000000662870
:080008000528A600030EA70065
:10001000A801A00A0A302002031D3428A001A10A69
:1000200006302102031D3428A101A20A0A3022024F
:10003000031D3428A201A30A06302302031D34281D
:10004000A301A40A03302402031930280A30240231
:10005000031D3428A401A50A02302502031D3428FB
:10006000251C3428A401A501851E3B28061E3E2818
:10007000861E4B285F28A001A1015F28A20A0A3032
:100080002202031D5F28A201A30A06302302031DDA
:100090005F28A3015F28A40A0330240203195A2809
:1000A0000A302402031D5F28A401A50A023025029C
:1000B000031D5F28251C5F28A401A5015F280C10E3
:1000C0008F17270E8300A60E260E090007309F000B
:1000D000831630308500F03086000C1483128501C1
:1000E00086010F309000C0308B008E018F01A80177
:1000F000A001A101A201A301A401A501A601A701DC
:1001000028140530A0000330A1000930A2000430FB
:10011000A3000130A4000130A500051485171221A9
:10012000051085141221851005151221051185155C
:1001300012218511851312210517051412210510AE
:10014000851412218510051512210511851512211E
:100150008511051312218615051412210510851429
:100160001221851005151221051185151221851101
:10017000861112210615051412210510851412216D
:1001800085100515122105118515122185110611FD
:1001900012218614051412210510851412218510D0
:1001A00005151221051185151221851186101221C0
:1001B0000614051412210510851412218510051549
:1001C0001221051185151221851106101221061024
:1001D00086100611861105138513200885008517E2
:1001E000851321088500051705132208850086154B
:1001F000861123088500061506112408850086143B
:100200008610250885000614051AE7288501860151
:100210006300051AE7280629FF30152964301529DF
:1002200032301529143015290130AB00C730A90030
:100230000130AA00A90B1D29AA0B1A29AB0B1629FC
:020240000800B4
:02400E00183D5B
:00000001FF
